:103C02000ECF0EBB0EA70E920E7C0E650E4D0E341D
:103C12000E190DFE0DE10DC40DA50D850D640D42AD
:103C22000D1E0CFA0CD40CAE0C860C5D0C330C0879
:103C32000BDC0BB00B820B540B250AF50AC40A935A
:103C42000A610A2F09FD09CA09960963092F08FCAE
:103C520008C808950861082E07FB07C8079607647D
:103C62000733070206D206A206730645061705EABF
:103C720005BF059305690540051704F004C904A3AF
:103C8200047E045A0437041503F403D303B40396E1
:103C92000378035B033F0324030A02F002D702BF47
:103CA20002A80292027C02670253023F022C021A0D
:103CB200020801F701E601D601C701B801A9019C7A
:103CC200018E018101740168015D01510146013CCF
:103CD20001320128011F0115010D010400FC00F44D
:103CE20000EC00E500DE00D700D000CA00C300BD32
:103CF20000B800B200AD00A700A2009E0099009497
:103D02000090008C008700840080007C00780075A1
:103D12000072006E006B0068006500620060005D6A
:103D2200005A0058005500530051004E004C004A02
:103D320000480046004400430041003F003E003C72
:103D4200003A0039003700360035003300320031C6
:103D5200002F002E002D002C002B002A0029002805
:103D62000027002600250024002300010C01010485
:103D720002011E030A9604013205020206006407CC
:103D8200010108000009015A0E01010F0001120091
:103D92006413010114013C1501FA1664FA17FFFFBE
:103DA2001D00072000072400022701012F013C30DB
:103DB200010132010335FFFF3603073CFFFF3DFFE0
:103DC200FF180002191E461A00021B00022D32C8FB
:103DD2002E0001FAFAFA18000019FFFF1A00001B60
:0B3DE20000002D32C82E0001FAFAFA92
:10004800900786E0FEA3E0FF7457BE0010D39F40E0
:100058000C903D6C12001EE493F599802F900014CB
:10006800E0D394044014900786E0FEA3E0FF903D9F
:100078006C12001EE493F5998012900786E0FEA3A7
:10008800E0FF903D8112001EE493F59990078612D7
:10009800000E900786E0FEA3E0FF746C6F4E7003BD
:1000A80075130022900072E0B40208740190007287
:1000B800F0D20C90013AE090002AF090013BE090D9
:1000C800002BF090013CE090002CF0A20AB34016FF
:1000D80090013AE0700C90013BE0700690013CE022
:1000E80060028002C20A90013AE0B4300F90013BEE
:1000F800E0B4470890013CE0643B60028004D20B06
:100108008002C20BE557B40102800302022E900060
:1001180057E0F565900062E0F567900063E0F568E8
:10012800900074E0F56990007AE0900029F0900062
:100138007CE0F56490007DE0F566900080E0F56372
:10014800900081E0F562900090E0900041F090000E
:1001580091E0900042F0900092E0900043F090000F
:1001680093E0900044F0900094E0900045F09000F7
:1001780095E0900046F0900096E0900047F09000DF
:1001880097E0900048F0900099E0900033F09000DC
:100198009AE0900034F090009BE0900035F09000D9
:1001A8009CE0900036F0900079E0B4011790000AC6
:1001B800740FF0A374FFF090000CE4F0A3F0740245
:1001C800900079F0900079E0B4035990000CE0FEBB
:1001D800A3E0FF90000AE0FCA3E0FD120003741006
:1001E800123F4D7408123F3FEF900026F0EF700663
:1001F80074FF900026F07400900079F090000BE0F6
:10020800900027F090000AE0900028F0900026E087
:10021800900789F0900027E090078AF0900028E086
:1002280090078BF0803F900081E07006755701754C
:100238006200A20AB3402E90013AE090002AF090A2
:10024800013BE090002BF090013CE090002CF090F6
:10025800002AE0700C90002BE0700690002CE06003
:10026800028002C20AE5657003756502E5677003DE
:100278007567027E887F4DE5658E048F05FF123F06
:100288002F8C388D39E56875F0FAA4FFAEF0E56774
:100298008E048F05FF123F2F8C3C8D3D90004FE060
:1002A800F55F90004DE0FE900069E0B506189000FB
:1002B8004CE0FE900068E0B5060C90004BE0FE9024
:1002C8000059E06E606F900069E07006900068E089
:1002D80060067400900059F0900069E0B40208903C
:1002E80000497401F08005900049E4F0900068E04E
:1002F800B4020890004A7401F0800590004AE4F0C6
:10030800900068E0600690004AE060028005755F32
:10031800038003755F04E558B55702D20C90006856
:10032800E090004CF0900069E090004DF09000598A
:10033800E090004BF0740190009EF0740090009FD4
:10034800F074009000A0F074009000A1F074009088
:1003580000A2F074009000A3F074009000A4F07460
:10036800019000A5F074009000A6F074009000A71A
:10037800F074009000A8F074009000A9F074009048
:1003880000AAF074009000ABF074019000ACF07417
:10039800009000ADF074009000AEF074009000AFD3
:1003A800F074009000B0F074009000B1F074009008
:1003B80000B2F07401900362F07400900363F0746B
:1003C80000900364F07400900365F0740090036675
:1003D800F07400900367F07400900368F074009064
:1003E80003A2F074009003A3F074009003A4F074C7
:1003F800009003A5F074009003A6F074009003A782
:10040800F074009003A8F074009003E2F074019077
:1004180003E3F074009003E4F074009003E5F074D3
:10042800009003E6F074009003E7F074009003E88E
:10043800F07401900422F07401900423F074009089
:100448000424F07400900425F07400900426F074DD
:1004580000900427F07400900428F022E5B554F7C2
:10046800F5B5E5B554FDF5B5C2A2C2A1C292C20761
:10047800E5B554FBF5B5755004E55004F551900009
:100488004FE0F55F900025E4F0C209E5B554FEF5AC
:10049800B522750A00750900AE09AF0A7457BE0087
:1004A800039F5003020557903D6C12001EE4939081
:1004B800004E123F650FBF00010EE0FC903D6C122C
:1004C800001EECFEE493FFEEC39F5026AE09AF0A70
:1004D8000FBF00010E903D6C12001EAE09AF0AE47A
:1004E80093FC903D6C12001EE49390004E123F6501
:1004F800ECF0AE09AF0A903D6C12001EE493900038
:100508004E123F65E0FC903D6E12001EECFCE49339
:10051800FDECD39D4019903D6E12001EE493FC90B3
:100528003D6C12001EE49390004E123F65ECF0AE55
:1005380009AF0A74022FFF50010E8E098F0A780A3C
:10054800740126F6500418E436F640030204A0228B
:10055800750A00750900AE09AF0A7415BE00039F3D
:100568005003020625903DC312001EE49390004EEE
:10057800123F650FBF00010EE0FC903DC312001E44
:10058800ECFEE493FFEEC39F5026AE09AF0A0FBFFF
:1005980000010E903DC312001EAE09AF0AE493FCA1
:1005A800903DC312001EE49390004E123F65ECF09C
:1005B800AE09AF0A903DC312001EE49390004E129C
:1005C8003F65E0FC903DC512001EECFCE493FDEC99
:1005D800D39D4019903DC512001EE493FC903DC385
:1005E80012001EE49390004E123F65ECF0AE09AF86
:1005F8000A740F6F4E7006750A15750900AE09AFBB
:100608000A74022FFF50010E8E098F0A780A7401AE
:1006180026F6500418E436F6400302055E22750AF1
:1006280000750900AE09AF0A7415BE00039F500398
:100638000206F3903DD812001EE49390004E123F3C
:10064800650FBF00010EE0FC903DD812001EECFEC5
:10065800E493FFEEC39F5026AE09AF0A0FBF000117
:100668000E903DD812001EAE09AF0AE493FC903DEF
:10067800D812001EE49390004E123F65ECF0AE09CC
:10068800AF0A903DD812001EE49390004E123F65C9
:10069800E0FC903DDA12001EECFCE493FDECD39DE7
:1006A8004019903DDA12001EE493FC903DD81200E8
:1006B8001EE49390004E123F65ECF0AE09AF0A7449
:1006C8000F6F4E7006750A15750900AE09AF0A74EA
:1006D800022FFF50010E8E098F0A780A740126F640
:1006E800500418E436F6400302062C22054C220575
:1006F8004B22054DC2CF2290F800E49364066002B5
:1007080080FE75840175A70075FF80900788E4F066
:1007180075C91075A70F75A1C775A70075D900759C
:10072800CEFF75A70F75F1FE75F2FF75F33775F4F7
:100738007875A4BA75A5FF75A60775AE0075AFFFE5
:1007480075D48175D5FF75D6FF75D7FFC296C2954A
:10075800C2A0C297E5B554BFF5B5E5B554DFF5B508
:10076800E5B554EFF5B5E5B5547FF5B5E5B554F7FE
:10077800F5B5E5B554FDF5B575A70075A20175A1E8
:100788004775F80975BC0175BE0475BD6C75BE0763
:1007980075BDA075BE0875BD0175BC0075BB187523
:1007A800BC2075BA0875E88075D11375A70F75E177
:1007B8000575E20075C740759700759780740A1231
:1007C8003F1F7597C0E5975420700280F8758F0217
:1007D80075A700D2AF75980075A90C75A70F75ABF2
:1007E8004375ADFB75AC1E75A700758911758E0034
:1007F800758C00758A00D2A9D28C758D00758B0016
:10080800D2ABD28E75CD0075CC0075CA0075CB0001
:10081800D2ADC2CFD2CA7591047592007593CD75C9
:10082800EF0675D94075CF01900786E4F0A3F075FF
:100838001300751400C299D20A74C8F51875170008
:1008480012252B75A70FE5FB90001AF0E5FA90002A
:100858001BF0E5F990001CF075A70090F800E493F0
:10086800F508122662122B9C900789E0900026F06A
:1008780090078AE0900027F090078BE0900028F01E
:1008880090078CE0900029F090078DE0F5659007BF
:100898008EE0F56790078FE0F568900790E0F569BE
:1008A800900791E0F564900792E0F566900793E071
:1008B800F563900794E0F562900795E090002AF0C0
:1008C800900796E090002BF0900797E090002CF0AE
:1008D800900798E0900041F0900799E0900042F06E
:1008E80090079AE0900043F090079BE0900044F056
:1008F80090079CE0900045F090079DE0900046F03E
:1009080090079EE0900047F090079FE0900048F025
:100918009007A0E0900033F09007A1E0900034F039
:100928009007A2E0900035F09007A3E0900036F021
:100938007400900082F090013AE0700C90013BE066
:10094800700690013CE060028004C20A8002D20A6C
:1009580090F807E493900021F0900021E0440A9079
:100968000021F0900021E054FE900021F0740690E0
:100978000012F07402900013F090F802E4939000D3
:1009880014F07403900015F07403900016F07401CD
:10099800900017F07405900018F0900014E0B4046B
:1009A800067404900018F0900014E0B40306740371
:1009B800900018F07404900019F090F804E49390F3
:1009C800001DF0740090001EF090F805E49390006C
:1009D8001FF090F806E493900020F074FF90002236
:1009E800F07447900125F0744D900126F074209022
:1009F8000127F07434900128F0744C900129F074A8
:100A08003890012AF0743090012BF0744590012C35
:100A1800F0742090012DF0742090012EF074209035
:100A2800012FF07434900130F07453900131F07458
:100A380050900132F07444900133F090007AE0D382
:100A480094014006740090007AF0755701755801BA
:100A5800740390004CF01200AC12049A900014E059
:100A6800B404051206268003120558122557E5B569
:100A780054FEF5B5900025E4F0900786E4F0A3F065
:100A880075230075220075470075290075280075C3
:100A9800480075310075300075490075530075546C
:100AA8000075590075500475510175333C75320055
:100AB800756F00756E007570CD75550075560075AB
:100AC8004200754300754400754500755A00754627
:100AD80000754100754000900006E4F0A3F0900016
:100AE80008E4F0A3F0755D00755E0090000E74FDDB
:100AF800F0A374E8F0900023E4F07464900024F00C
:100B0800C200D201C202D203754C00756C00C294B7
:100B1800C293C287C290C291C20C7E017F0090002E
:100B280028E0123F4D900027E02FFF50010E900063
:100B38000AEEF0A3EFF0900026E0700674FF900034
:100B480026F090000AE0FEA3E0FFEFD394FFEE94B6
:100B58000F400790000AE4F0A3F07400900071F0D1
:100B68007400900079F07400900082F07400900096
:100B78008DF074009000B4F0E56670037566047437
:100B88003A90074EF074FD90074FF09003D4E09030
:100B98000414F0D2B0D2B7D2A7D2A6D2B1D2A3C28F
:100BA80007A2B6B39204A2B3B39205D29CD2EC7555
:100BB800CF01A298B34005C298122F00E513600632
:100BC800A299B3B340028005C299123476E5146441
:100BD800016005E514B4040280D5E54CD3940540C2
:100BE8000CE559C394C850020559754C00E570C30B
:100BF80094FA501A786E12003FAE6EAF6FEFD3942E
:100C0800E8EE940340080570756F00756E00C28E9B
:100C18007E047F00E54B123F4DE58D75F004A4FD81
:100C2800ACF0EF2DFDEE3CFCE58B75F04084FF7ECB
:100C380000ED2FFFEC3EFE8E248F25D28EA2B6301B
:100C48000401B35003020D7DA2B6300401B3500372
:100C5800020D7DA2B6405A0553E5B54401F5B5909D
:100C68000024E4F0E553D3956540447C887D4D121B
:100C78003DED8E228F23E5472FFF50010E740112A0
:100C88003F3F8E228F23852347755301C28E758D72
:100C980000758B00754B00D28E7403BE00039F5005
:100CA800069000257401F0E542B40603754200D2AF
:100CB80004A2B6B35003020D7DC20490006BE0603D
:100CC800181235B7A200B34008E5B54408F5B58059
:100CD80006E5B554F7F5B58002C20090006EE060F5
:100CE8001812370CA202B34008E5B54402F5B580E6
:100CF80006E5B554FDF5B58006E5B554FDF5B5A294
:100D080007B34004D2878002C287900059E060048C
:100D1800D2908002C29090004AE0B40104D294803C
:100D280002C294900049E0B40104D2938002C293B5
:100D3800A209B34004D2918002C291900018E0FE4B
:100D4800900014E0C39E4009900014E0D39408403A
:100D58000974FB900023F012046490001DE06015F4
:100D680090001DE0FE900017E06E600974FE900090
:100D780023F0120464C2CA7E017F00E54D123F4D84
:100D8800E5CD2FFF50010E8E268F27D2CAE564B419
:100D9800014890000EE0FCA3E0FDEFC39DEE9C40EF
:100DA80039B208E52945286013A208B34008E5B51B
:100DB8004404F5B58006E5B554FBF5B590000EE0A2
:100DC800FEA3E0FF900010E0FCA3E0FDEF2DFDEE98
:100DD8003CFC90000EECF0A3EDF0A2B3300501B39B
:100DE8005003020EC2A2B3300501B35003020EC273
:100DF800A2B35003020EBB0554E5B54401F5B59006
:100E08000024E4F0E554D395675003020EB97CEA58
:100E18007D60AE26AF27123DED8E288F29E568123A
:100E28003F4D74FF8E048F05FF123F2F8C288D29AC
:100E3800E5482DFD50010C74018C068D07123F3FCB
:100E48008E288F29852948A209B340157464123F5A
:100E58004D900067E08E048F05FF123F2F8C288D80
:100E68002975540190000EE0FEA3E0FFAC26AD27E3
:100E780012000390000EEEF0A3EFF0E566FF123FBC
:100E88002F740AFF123F2F90007BE08C068D07120B
:100E98003F4D74148E048F05FF123F2F900010EC05
:100EA800F0A3EDF0C2CA75CD0075CC00754D00D227
:100EB800CAD205A2B3B34002C205900025E0B4012E
:100EC80007E555C3940640030214D3E56C90250A40
:100ED800F8282873900059E0C394024003021030A8
:100EE800E550D394015003021030E55075F040A44A
:100EF800FFAEF090031212001EE0C395445018E5AF
:100F08005075F040A4FFAEF090031112001EE0F5FA
:100F18002D752C00021030E55075F040A4FFAEF09E
:100F280090031012001EE0C395444003020FCCE565
:100F38005075F040A4FFAEF090031112001EE5506A
:100F480075F040A4FFAEF0E0FC90030F12001EEC19
:100F5800FEE0FFEEC39FFEE5508E0475F040A4FF4F
:100F6800AEF090031012001EE0F40425448C0088B3
:100F7800F0A4FFAEF0E5508F048E0575F040A4FF95
:100F8800AEF090031212001EE55075F040A4FFAEBB
:100F9800F0E0FA90031012001EEAFEE0FFEEC39F95
:100FA800FECDCCCD8E07123F2FE55075F040A4FF43
:100FB800AEF090030F12001EE02DFD50010C8C2C9A
:100FC8008D2D8064E55075F040A4FFAEF090030FBE
:100FD80012001EE55075F040A4FFAEF0E0FC90034F
:100FE8000E12001EECFEE0FFEEC39F8544F0A4FF46
:100FF800AEF0E5508F048E0575F040A4FFAEF0907A
:10100800031012001EE0FECDCCCD8E07123F2FE557
:101018005075F040A4FFAEF090030E12001EE02DB4
:10102800FD50010C8C2C8D2D756C010214D3900091
:1010380059E0C3940240030211E390004FE0D395B6
:1010480050500302118CE55075F040A4FFAEF090AB
:10105800031812001EE0C395445018E55075F0407F
:10106800A4FFAEF090031712001EE0F52B752A00BE
:1010780002118CE55075F040A4FFAEF090031612F3
:10108800001EE0C395444003021128E55075F04066
:10109800A4FFAEF090031712001EE55075F040A4AF
:1010A800FFAEF0E0FC90031512001EECFEE0FFEE30
:1010B800C39FFEE5508E0475F040A4FFAEF0900388
:1010C8001612001EE0F40425448C0088F0A4FFAE3C
:1010D800F0E5508F048E0575F040A4FFAEF0900344
:1010E8001812001EE55075F040A4FFAEF0E0FA902B
:1010F800031612001EEAFEE0FFEEC39FFECDCCCD24
:101108008E07123F2FE55075F040A4FFAEF0900314
:101118001512001EE02DFD50010C8C2A8D2B8064C9
:10112800E55075F040A4FFAEF090031512001EE5DF
:101138005075F040A4FFAEF0E0FC90031412001EBE
:10114800ECFEE0FFEEC39F8544F0A4FFAEF0E5504F
:101158008F048E0575F040A4FFAEF09003161200C0
:101168001EE0FECDCCCD8E07123F2FE55075F04026
:10117800A4FFAEF090031412001EE02DFD50010CE8
:101188008C2A8D2BE550B40122E55FD39401401BD6
:10119800E550C395555014E544C39405500D90038C
:1011A8005FE0A828B8000695294002800375500220
:1011B800E550B55F2290004FE0D395504019E550B7
:1011C80075F040A4FFAEF090031712001EE0A822AD
:1011D800B80006952340028002055F756C02021470
:1011E800D3900059E0B4022AE55075F040A4FFAE50
:1011F800F090031712001EE0F52B752A00E55075D4
:10120800F040A4FFAEF090030E12001EE0F52D751D
:101218002C00900059E0B4030F900051E0F52B75B5
:101228002A00752D00752C00756C030214D3E55047
:1012380075F040A4FFAEF090032012001EE0C395A5
:1012480059400302130A900049E07036E550D394E0
:10125800014029AE22AF23AC2CAD2DEDD39FEC9EDF
:10126800401AE55075F040A4FFAEF090031E12003E
:101278001EE0A828B80005D3952950028002155011
:101288008034E550D394024029AE22AF23AC2CAD74
:101298002DEDD39FEC9E401AE55075F040A4FFAEAB
:1012A800F090031E12001EE0A828B80005D3952967
:1012B800500280021550E550B55136E550C3955F90
:1012C800502FE550C395555028AE22AF23AC2AAD18
:1012D8002BEFD39DEE9C4019E55075F040A4FFAE6E
:1012E800F090031F12001EE0A828B80006952940B8
:1012F8000280020550C292E55065516005C207752B
:101308005900756C040214D3E55075F040A4FFAE83
:10131800F090031A12001EE0B40117E55075F04072
:10132800A4FFAEF090032012001EE0240AC39559D2
:1013380040030213E0752F64752E00A207B3500B0B
:10134800900060E02405C3954440030213E0E55093
:1013580075F040A4FFAEF090031D12001EE0C39587
:10136800444064E55075F040A4FFAEF090031C12B1
:10137800001EE55075F040A4FFAEF0E0FC90031BA2
:1013880012001EECFEE0FFEEC39F8544F0A4FFAE02
:10139800F0E5508F048E0575F040A4FFAEF0900381
:1013A8001D12001EE0FECDCCCD8E07123F2FE5505A
:1013B80075F040A4FFAEF090031B12001EE02DFD57
:1013C80050010C8C2E8D2FAE22AF23AC2EAD2FEFFB
:1013D800D39DEE9C4002D207756C050214D3E550EC
:1013E800B40109900059E0C3940240030214B39079
:1013F8000358E0D3954450030214B3900356E0C356
:1014080095445040900357E0FE900355E0F4042EB5
:10141800FE900356E0F40425448E0088F0A4FFAE45
:10142800F0900358E0FC900356E0F4042C8E048FEF
:1014380005FF123F2F900355E02DFD50010C8C2A1B
:101448008D2B802C900355E0FE900354E0F4042E7D
:101458008544F0A4FFAEF0900356E08E048F05FF9C
:10146800123F2F900354E02DFD50010C8C2A8D2B38
:10147800E550C3955F502FE550C395555028AE22CF
:10148800AF23AC2AAD2BEFD39DEE9C4019E55075E8
:10149800F040A4FFAEF090031F12001EE0A828B889
:1014A8000006952940028003755002900049E0B477
:1014B8000106E550640160028003755002E550653D
:0B14C800516005C207755900756C00EB
:10250A00020EDC0210360211E90212360213100220
:02251A0013E6C6
:1014D300900050E02402A822B80007D395234002CD
:1014E300C207900025E0B40109900059E0C39403BA
:1014F3004003021659900049E060030215A9E55024
:10150300D394014034E55075F040A4FFAEF090034E
:101513001412001EE0A822B8001FD39523401AE539
:101523005075F040A4FFAEF090031F12001EE0A818
:1015330028B80005D39529500280021550E550D3F1
:101543009401402FE55075F040A4FFAEF0900312D4
:1015530012001EE0C39544501AE55075F040A4FFF5
:10156300AEF090031E12001EE0A828B80005D39524
:1015730029500280021550E550D394014021E550D3
:10158300D39555401AE55075F040A4FFAEF0900393
:101593001E12001EE0A828B80005D395295002802A
:1015A30002155002164EE550D394024034E55075AF
:1015B300F040A4FFAEF090031412001EE0A822B87E
:1015C300001FD39523401AE55075F040A4FFAEF0F9
:1015D30090031F12001EE0A828B80005D3952950D8
:1015E3000280021550E550D39402402FE55075F068
:1015F30040A4FFAEF090031212001EE0C3954450C6
:101603001AE55075F040A4FFAEF090031E12001EC1
:10161300E0A828B80005D39529500280021550E5AB
:1016230050D394024021E550D39555401AE55075A7
:10163300F040A4FFAEF090031E12001EE0A828B8ED
:101643000005D39529500280021550E5506551607D
:1016530005C207755900900060E0D3954450099086
:101663000054E0C395445002C207900059E0700350
:101673000218BCA2A5B34008A2A4B340030218A554
:10168300AE34AF357441D39F749C9E4005783412B9
:10169300003FAE34AF35EFB48806EEB413028003D7
:1016A300021882A2A55003021745900059E0B40125
:1016B3000B90004FE0D3955F4002055F900059E027
:1016C300B40253E55075F040A4FFAEF0900320122E
:1016D300001EE0C39559503E90004FE0D395504013
:1016E30020E550C395555019E55075F040A4FFAE61
:1016F300F090031412001EE0A822B80006952340C0
:10170300028002055090004FE0F55FE5506551609F
:1017130005C207755900900059E0B4032590004FA6
:10172300E0D395504007E550C3955540028002052C
:101733005090004FE0F55FE55065516005C20775B5
:101743005900A2A45003021882900059E0B4016E1C
:10175300900049E07035E550D394014029E5507578
:10176300F040A4FFAEF090031E12001EE0A828B8BC
:10177300000FD39529400A155075590085505F8095
:101783000385505F8003755F018033E550D3940276
:101793004029E55075F040A4FFAEF090031E1200FF
:1017A3001EE0A828B8000FD39529400A1550755993
:1017B3000085505F800385505F8003755F02900052
:1017C30059E0D394015003021876E55075F040A414
:1017D300FFAEF090032012001EE0C39559400302B0
:1017E3001876900049E07041E550D394014034E508
:1017F3005075F040A4FFAEF090031112001EE0A854
:1018030022B8001FD39523401AE55075F040A4FF7A
:10181300AEF090031E12001EE0A828B80005D39571
:1018230029500280021550803FE550D39402403482
:10183300E55075F040A4FFAEF090031112001EE0D6
:10184300A822B8001FD39523401AE55075F040A491
:10185300FFAEF090031E12001EE0A828B80005D3C7
:101863009529500280021550E55065516005C20765
:10187300755900E555B40704055D8003755D00E502
:1018830062B4010EAE34AF35EF64407005EE649C74
:101893006002800EA2A54003755701A2A440037500
:1018A3005702A2A5B3B35006A2A4B3B34002800665
:1018B3007535007534000219AAA2A5B34008A2A485
:1018C300B34003021996AE34AF357441D39F749C71
:1018D3009E4005783412003FAE34AF35EFB488062E
:1018E300EEB413028003021996A2A5406F9000681C
:1018F300E0605A90004AE0B4010790004AE4F080A7
:101903000690004A7401F090004AE07005755F0389
:101913008003755F0490004AE0B40104D29480020E
:10192300C294E550B4041AE55075F040A4FFAEF03C
:1019330090031E12001EE0A828B80005D395295075
:10194300028008755003C2077559008003755F0450
:10195300E555B40704055D8003755D00A2A440331B
:10196300900069E06021900049E0B40107900049CC
:10197300E4F080069000497401F0900049E0B4015E
:1019830004D2938002C293E555B40704055D800336
:10199300755D00A2A5B3B35006A2A4B3B340028001
:1019A30006753500753400E557655860069000826A
:1019B300E06003021B32C29C751400751300C2CA97
:1019C300E55790251CF82828738012122B9C800D54
:0D19D300122C758008122D4E8003122E2755
:0F251C000219CC0219CE0219D30219D80219DD07
:1019E000900029E090007AF0E565900057F0E567F7
:1019F000900062F0E568900063F0E569900074F093
:101A0000E56490007CF0E56690007DF0E563900071
:101A100080F0E562900081F090002AE090013AF0B9
:101A200090002BE090013BF090002CE090013CF006
:101A3000900041E0900090F0900042E0900091F022
:101A4000900043E0900092F0900044E0900093F00A
:101A5000900045E0900094F0900046E0900095F0F2
:101A6000900047E0900096F0900048E0900097F0DA
:101A7000900033E0900099F0900034E090009AF0EC
:101A8000900035E090009BF0900036E090009CF0D4
:101A90007400900082F07447900125F0744D90011D
:101AA00026F07420900127F07434900128F0744CD3
:101AB000900129F0743890012AF0743090012BF0D5
:101AC000744590012CF0742090012DF07420900149
:101AD0002EF0742090012FF07434900130F0745384
:101AE000900131F07450900132F07444900133F061
:101AF0009003D4E0900414F0743A90074EF074FD13
:101B000090074FF01200AC900004E4F0A3F09000B6
:101B1000067475F0A37430F09000087475F0A37427
:101B200030F0855758D2CA754B00D29C741B900078
:101B300023F0E555C394065005E550B55102804E9B
:101B4000C207E55075F040A4FFAEF09003221200EA
:101B50001EE030E003D38001C39296E55075F0405B
:101B6000A4FFAEF090032312001EE030E003D38008
:101B700001C39295855051AE28AF297405BE00036C
:101B80009F5007E544D3940550028002D292E55558
:101B9000D394055003021C57C207E550D39401406B
:101BA00059E55075F040A4FFAEF090031E12001EE0
:101BB000E0A828B80007D3952940021550E55065E4
:101BC000516035E55075F040A4FFAEF0900322124D
:101BD000001EE030E003D38001C39296E55075F01B
:101BE00040A4FFAEF090032312001EE030E003D3C8
:101BF0008001C39295855051805DE555B4061A90D9
:101C000000ACE030E003D38001C392969000ADE0D9
:101C100030E003D38001C39295E555B4071A9000D4
:101C2000A5E030E003D38001C392969000A6E03097
:101C3000E003D38001C39295E555B4081A90009E45
:101C4000E030E003D38001C3929690009FE030E043
:101C500003D38001C39295900072E06058E544750B
:101C6000F00284FF7E0090014E12001EE0F55BE55D
:101C70004675F00A84FF7E0090024E12001EE0F5C9
:101C80005CE55B255CD39464400BE55B255CC39409
:101C900064F55B8003755B00E55B75F00284FF7E95
:101CA000008F5BEFC394335007EF24CDF55B8003C7
:101CB000755BFF801CE54475F00284FF7E00900197
:101CC0004E12001EE075F00284FF7E00EF24CDF579
:101CD0005BE595C3955B4004C2A28002D2A2A20735
:101CE000B34005E555B407037570CDE595C3957010
:101CF0004004C2A18002D2A1E542C394064003027F
:101D000022FBA2EDB350030222FBC2EDE5426003C9
:101D1000021E5D7E017F00E5BE123F4DE5BD2FFF37
:101D200050010E900000EEF0A3EFF0900029E0B417
:101D300001177E0F7FFF900000E0FCA3E0FD120082
:101D400003900000EEF0A3EFF0900079E0B4025BA6
:101D5000900000E0FEA3E0FF90000AE0FCA3E0FD9D
:101D6000EDD39FEC9E400F900000E0F8A3E09000C0
:101D70000AC8F0A3C8F0900000E0FEA3E0FF9000C6
:101D80000CE0FCA3E0FDEFD39DEE9C400F90000023
:101D9000E0F8A3E090000CC8F0A3C8F0900000E0C9
:101DA000FEA3E0FF7404123F3F8F43900079E07080
:101DB00060900000E0FEA3E0FF90000AE0FCA3E0DA
:101DC000FDEFD39DEE9C400D120003900000EEF05D
:101DD000A3EFF08007900000E4F0A3F0900000E093
:101DE000FEA3E0FF7410123F4D900026E08E048F9A
:101DF00005FF123F2F900000ECF0A3EDF07400D32C
:101E00009D74019C4008900001E0F54380037543F8
:101E1000FFE54375F00AA4FFAEF074198E048F0538
:101E2000FF123F2F8D44ED2531FFAE3050010E746F
:101E300001123F3F8F44854431753000EFD39462E7
:101E40004003754462900072E06401600690006691
:101E5000E060028005754201800375BB17E542B45E
:101E600001028003021F4D7E017F00E5BE123F4D3F
:101E7000E5BD2FFF50010E900000EEF0A3EFF090B3
:101E80000072E0B4017EE53345326025AC32AD33FB
:101E90001DBDFF011C8F028E038C068D07903C0236
:101EA00012002EE493FE740193FFEFC39AEE9B4061
:101EB0000280057832123F77AE32AF3374B3BE0082
:101EC00025D39F4021900000E0FCA3E0FD0FBF0060
:101ED000010E903C0212002EE493FE740193FFED7C
:101EE000C39FEC9E40028005783212003FAE32AFB5
:101EF00033E569123F4D74648E048F05FF123F2F46
:101F00008D468033900066E0602D900000E0FEA3D7
:101F1000E0FFEFD39400EE9408400F900066E0B429
:101F20000104C2098002D209800D900066E0B4016C
:101F300004D2098002C209900072E0640260069037
:101F40000066E0600575BB168003754202E542B489
:101F50000202800302203B7E017F00E5BE123F4D5E
:101F6000E5BD2FFF50010E900000EEF0A3EFF090C2
:101F70000072E0B4027EE53345326025AC32AD3309
:101F80001DBDFF011C8F028E038C068D07903A98B1
:101F900012002EE493FE740193FFEFC39AEE9B4070
:101FA0000280057832123F77AE32AF3374B3BE0091
:101FB00025D39F4021900000E0FCA3E0FD0FBF006F
:101FC000010E903A9812002EE493FE740193FFEDF7
:101FD000C39FEC9E40028005783212003FAE32AFC4
:101FE00033E569123F4D74648E048F05FF123F2F55
:101FF0008D468033900066E0602D900000E0FEA3E7
:10200000E0FFEFD39400EE9408400F900066E0B438
:102010000104C2098002D209800D900066E0B4017B
:1020200004D2098002C209900072E0700375460074
:10203000900066E07002C20975BB1FE542B403451B
:102040007E017F00E5BE123F4DE5BD2FFF50010E22
:10205000900000EEF0A3EFF07409123F4D74E68E8D
:10206000048F05FF123F2F8C408D41E5492DFD5017
:10207000010C74018C068D07123F3F8E408F418505
:10208000414975BB19E542B4040280030221E37E95
:10209000017F00E5BE123F4DE5BD2FFF50010E90C0
:1020A0000000EEF0A3EFF07404123F3F8F4AE563A7
:1020B000B401028003022170756A00756A00E56A46
:1020C000D39407400302215DE56A900041123F6509
:1020D000E0D3954A501AE56A900041123F65E0F45A
:1020E00004254AFEE56A900037123F65EEF080173E
:1020F000E56A900041123F65E0C3954AFEE56A90AB
:102100000037123F65EEF0E56AC394044009900081
:1021100084E0C3956A503BE56A6029E56A90003720
:10212000123F65FEE0FFEE90003FE0D39F4013E5D5
:102130006A900037123F65E090003FF0E56A90003A
:1021400040F0800E900037E090003FF07400900067
:1021500040F0786A740126F640030220BE900040E9
:10216000E0F4042408F555E555D394054002C292E5
:10217000E563D39401402FE54AD3946E4004D20D19
:102180008002C20D755505E563B40205A20DB3408A
:10219000028003755507E563B40306A20DB3B3408F
:1021A000028003755507E55665556008E55004F54E
:1021B00051855556E555B40708E5B54480F5B58019
:1021C00006E5B5547FF5B5E55564066005E555B4FB
:1021D0000808E5B54410F5B58006E5B554EFF5B54A
:1021E00075BB13E542B4050280030222F77E017F2E
:1021F00000E5BE123F4DE5BD2FFF50010E900000DF
:10220000EEF0A3EFF07404123F3F8F45E562B40295
:102210000280030222F4756A00756A00E56AD394AD
:102220000340030222ABE56A900033123F65E0D31E
:102230009545501AE56A900033123F65E0F4042595
:1022400045FEE56A90002D123F65EEF08017E56AC5
:10225000900033123F65E0C39545FEE56A90002D7E
:10226000123F65EEF0E56A6029E56A90002D123FA5
:1022700065FEE0FFEE900031E0D39F4013E56A90E9
:10228000002D123F65E0900031F0E56A900032F0D9
:10229000800E90002DE0900031F07400900032F03C
:1022A000786A740126F6400302221C900082E070D6
:1022B00043E52945286036E557C39403500A90004A
:1022C00032E004C3940340028007900032E004F53A
:1022D00057E557D39402400A900032E004D39402A9
:1022E00050028007900032E004F5578007900032DA
:1022F000E004F55775BB180542D2ECE55DD39404B4
:1023000050030223E375CF01C2A2AE34AF35748807
:10231000D39F74139E4005A2A5B34014AE34AF35CD
:102320007488D39F74139E4005A2A4B340028048D2
:10233000783412003FAE34AF35EFB4883BEEB413BF
:1023400037A2A5B3500990004FE0D39550500280BA
:102350000405508011A2A5B3500890004FE06550CD
:1023600060028002D207A2A4B35007E550D39401C3
:10237000500280041550C207A2A5B3B35006A2A410
:10238000B3B340028006753500753400E5506551E1
:102390006035E55075F040A4FFAEF09003221200C6
:1023A0001EE030E003D38001C39296E55075F04003
:1023B000A4FFAEF090032312001EE030E003D380B0
:1023C00001C39295855051A20740057570CD8003D9
:1023D0007570FFE595C395704004C2A18002D2A13B
:1023E000022305AE24AF25EFD39420EE944E500384
:1023F0000224DE120464C28E758D00758B00754B4D
:1024000000D28EC207756F00756E007570CD755065
:1024100004752300752200755300755900C287901A
:102420000059E06004D2908002C29090004AE0B46B
:102430000104D2948002C294900049E0B40104D215
:10244000938002C293A209B34004D2918002C29148
:1024500090006BE060181235B7A200B34008E5B5F4
:102460004408F5B58006E5B554F7F5B58002C2001D
:1024700090006EE0601812370CA202B34008E5B578
:102480004402F5B58006E5B554FDF5B58006E5B521
:1024900054FDF5B590000E74FDF0A374E8F0E5422C
:1024A000B40603754200900025E4F07525007524FC
:1024B00000758D00758B00754B00900024E0C3946F
:1024C000035008900024E004F08006740390002478
:1024D000F0900024E0B40306E5B554FEF5B5AE2651
:1024E000AF27EFD39410EE9427401CC2CA75CD00DD
:1024F00075CC00752700752600D2CA754D00752968
:0A25000000752800755400020BB7A7
:1038BE00000001000132016401960196020002121D
:1038CE0002240200020003000340038003C0040030
:1038DE000440048004C00500060006000600060031
:1038EE00060006000600060000FF01310163019587
:1038FE0001FF01FF0211022302FF02FF02FF033F3D
:10390E00037F03BF03FF043F047F04BF04FF05FFD3
:10391E0006FF06FF06FF06FF06FF06FF06FF06FF71
:10392E000FAA0FA50F9F0F9A0F940F8D0F870F8061
:10393E000F780F710F680F600F570F4E0F450F3B2B
:10394E000F300F250F1A0F0E0F020EF50EE80EDBBD
:10395E000ECC0EBE0EAE0E9F0E8E0E7D0E6C0E5A41
:10396E000E470E340E200E0C0DF70DE20DCB0DB5DD
:10397E000D9D0D850D6D0D540D3A0D200D050CE9A7
:10398E000CCE0CB10C940C760C580C3A0C1B0BFB99
:10399E000BDB0BBB0B9A0B790B570B350B130AF189
:1039AE000ACE0AAB0A870A640A400A1C09F809D42F
:1039BE0009B0098C09670943091F08FB08D608B22C
:1039CE00088E086A0846082307FF07DC07B9079622
:1039DE0007730751072F070D06EC06CA06AA0689BC
:1039EE0006690649062A060A05EC05CD05B00592BC
:1039FE0005750558053C0520050504EA04CF04B5F8
:103A0E00049C04820469045104390422040B03F457
:103A1E0003DE03C803B2039D038903750361034DDF
:103A2E00033B03280316030402F202E102D102C093
:103A3E0002B002A00291028202730265025702498D
:103A4E00023C022F02220216020901FD01F201E6DA
:103A5E0001DB01D001C601BB01B101A7019D01949B
:103A6E00018B0182017901700168016001580150DA
:103A7E000148014101390132012B0125011E0118B6
:103A8E000111010B010500FF00FA0FA60FA00F99FF
:103A9E000F920F8B0F840F7C0F740F6B0F620F58EA
:103AAE000F4E0F430F380F2C0F1F0F120F050EF76F
:103ABE000EE80ED80EC80EB70EA50E930E800E6C25
:103ACE000E580E420E2C0E150DFD0DE40DCB0DB144
:103ADE000D950D790D5D0D3F0D200D010CE10CC006
:103AEE000C9E0C7C0C590C350C100BEA0BC40B9E67
:103AFE000B760B4F0B260AFD0AD40AAA0A800A552A
:103B0E000A2A09FF09D409A8097C0950092508F9D0
:103B1E0008CD08A10875084A081E07F307C8079DB7
:103B2E0007730749072006F706CE06A6067E065738
:103B3E000630060A05E405BF059B057705540532D8
:103B4E00051004EF04CE04AE048F04710453043543
:103B5E00041903FD03E203C703AD0394037B036360
:103B6E00034B0334031E030802F302DE02CA02B63D
:103B7E0002A30291027F026D025C024C023C022CF7
:103B8E00021D020E020001F201E401D701CA01BEBC
:103B9E0001B101A6019A018F0185017A01700166BA
:103BAE00015D0153014A0141013901310129012110
:103BBE0001190112010B010400FD00F700F000EAEB
:103BCE0000E400DE00D900D300CE00C900C400BF5F
:103BDE0000BA00B500B100AD00A800A400A0009C82
:103BEE00009900950091008E008A00870084008164
:043BFE00007E007BCA
:10252B00751A00751900AE19AF1AAC17AD18EDC3BB
:10253B009FEC9E401674FF123F1F75CF01781A74E3
:10254B000126F6500418E436F650DB22900786E499
:10255B00F0A3F0751000750F00751300751400C211
:10256B000ED20F22C2AF75D900758F0375B7A57543
:10257B00B7F190F800E4F0758F0175B7A575B7F159
:10258B00E50890F800F075B7A575B7F190F801E480
:10259B00F075B7A575B7F190079DE090F802F0754F
:1025AB00B7A575B7F19007A1E090F803F075B7A543
:1025BB0075B7F190079EE090F804F075B7A575B765
:1025CB00F190079FE090F805F075B7A575B7F190FE
:1025DB0007A0E090F806F075B7A575B7F19007A2C4
:1025EB00E090F807F0758F0075D940D2AF229007B5
:1025FB0088E0B4AB61C2AF75D90075B62275F52210
:10260B00758F0375B7A575B7F1740090F600F0756B
:10261B008F01750A00750900AE09AF0A7413BE006D
:10262B00279F402475B7A575B7F190078912001E37
:10263B00E0FC90F60012001EECF0780A740126F60E
:10264B00500418E436F650D0758F0075F51175B639
:10265B002075D940D2AF22C2AF75D90075F522755E
:10266B000A00750900AE09AF0A7413BE00229F4021
:10267B001F90F60012001EE493FC90078912001EB7
:10268B00ECF0780A740126F6500418E436F650D5AF
:10269B0075F51175D940D2AF22900788E0B4AA0224
:1026AB0080030227E1C2AF75D90075B62275F522FA
:1026BB00758F0375B7A575B7F1740090EE00F075C3
:1026CB00B7A575B7F1740090F000F075B7A575B7A5
:1026DB00F1740090F200F075B7A575B7F174009026
:1026EB00F400F0758F01750A00750900AE09AF0A89
:1026FB0074FFC39F74019E402475B7A575B7F19005
:10270B00004E12001EE0FC90EE0012001EECF07862
:10271B000A740126F6500418E436F650CF750A00F9
:10272B00750900AE09AF0A74FFC39F74019E402464
:10273B0075B7A575B7F190024E12001EE0FC90F034
:10274B000012001EECF0780A740126F6500418E40F
:10275B0036F650CF750A00750900AE09AF0A74FF43
:10276B00C39F74019E402475B7A575B7F190044EB5
:10277B0012001EE0FC90F20012001EECF0780A74BE
:10278B000126F6500418E436F650CF750A00750989
:10279B0000AE09AF0A74FFC39F74019E402475B746
:1027AB00A575B7F190064E12001EE0FC90F40012D6
:1027BB00001EECF0780A740126F6500418E436F685
:1027CB0050CF758F0075F51175B62075D940D2AF06
:1027DB00743A90074EF022900788E0B4AA02800367
:1027EB0002291FC2AF75D90075B62275F522758FF8
:1027FB000375B7A575B7F1740090E600F075B7A532
:10280B0075B7F1740090E800F075B7A575B7F17462
:10281B000090EA00F075B7A575B7F1740090EC0065
:10282B00F0758F01750A00750900AE09AF0A74FFC8
:10283B00C39F74019E402475B7A575B7F190004EE8
:10284B0012001EE0FC90E60012001EECF0780A74F9
:10285B000126F6500418E436F650CF750A007509B8
:10286B0000AE09AF0A74FFC39F74019E402475B775
:10287B00A575B7F190024E12001EE0FC90E8001215
:10288B00001EECF0780A740126F6500418E436F6B4
:10289B0050CF750A00750900AE09AF0A74FFC39FCC
:1028AB0074019E402475B7A575B7F190044E1200C4
:1028BB001EE0FC90EA0012001EECF0780A74012670
:1028CB00F6500418E436F650CF750A00750900AEC1
:1028DB0009AF0A74FFC39F74019E402475B7A57599
:1028EB00B7F190064E12001EE0FC90EC0012001E99
:1028FB00ECF0780A740126F6500418E436F650CF43
:10290B00758F0075F51175B62075D940D2AF743A35
:10291B0090074EF022900788E0B4AA028003022AA7
:10292B005DC2AF75D90075B62275F522758F03752B
:10293B00B7A575B7F1740090DE00F075B7A575B744
:10294B00F1740090E000F075B7A575B7F1740090C5
:10295B00E200F075B7A575B7F1740090E400F0755F
:10296B008F01750A00750900AE09AF0A74FFC39F8A
:10297B0074019E402475B7A575B7F190004E1200F7
:10298B001EE0FC90DE0012001EECF0780A740126AB
:10299B00F6500418E436F650CF750A00750900AEF0
:1029AB0009AF0A74FFC39F74019E402475B7A575C8
:1029BB00B7F190024E12001EE0FC90E00012001ED8
:1029CB00ECF0780A740126F6500418E436F650CF72
:1029DB00750A00750900AE09AF0A74FFC39F740135
:1029EB009E402475B7A575B7F190044E12001EE0FA
:1029FB00FC90E20012001EECF0780A740126F650EF
:102A0B000418E436F650CF750A00750900AE09AF0D
:102A1B000A74FFC39F74019E402475B7A575B7F167
:102A2B0090064E12001EE0FC90E40012001EECF02B
:102A3B00780A740126F6500418E436F650CF758FD9
:102A4B000075F51175B62075D940D2AF743A900761
:102A5B004EF022900788E0B4AA028003022B9BC29F
:102A6B00AF75D90075B62275F522758F0375B7A5AD
:102A7B0075B7F1740090D600F075B7A575B7F17402
:102A8B000090D800F075B7A575B7F1740090DA0017
:102A9B00F075B7A575B7F1740090DC00F0758F0178
:102AAB00750A00750900AE09AF0A74FFC39F740164
:102ABB009E402475B7A575B7F190004E12001EE02D
:102ACB00FC90D60012001EECF0780A740126F6502A
:102ADB000418E436F650CF750A00750900AE09AF3D
:102AEB000A74FFC39F74019E402475B7A575B7F197
:102AFB0090024E12001EE0FC90D80012001EECF06B
:102B0B00780A740126F6500418E436F650CF750A8D
:102B1B0000750900AE09AF0A74FFC39F74019E4094
:102B2B002475B7A575B7F190044E12001EE0FC900A
:102B3B00DA0012001EECF0780A740126F650041825
:102B4B00E436F650CF750A00750900AE09AF0A746A
:102B5B00FFC39F74019E402475B7A575B7F190060E
:102B6B004E12001EE0FC90DC0012001EECF0780A06
:102B7B00740126F6500418E436F650CF758F0075A5
:102B8B00F51175B62075D940D2AF743A90074EF057
:102B9B0022C2AF75D90075F522750A00750900AE12
:102BAB0009AF0A74FFC39F74019E401F90EE001281
:102BBB00001EE493FC90004E12001EECF0780A7499
:102BCB000126F6500418E436F650D4750A00750940
:102BDB0000AE09AF0A74FFC39F74019E401F90F0B3
:102BEB000012001EE493FC90024E12001EECF078D3
:102BFB000A740126F6500418E436F650D4750A0010
:102C0B00750900AE09AF0A74FFC39F74019E401F84
:102C1B0090F20012001EE493FC90044E12001EEC86
:102C2B00F0780A740126F6500418E436F650D47581
:102C3B000A00750900AE09AF0A74FFC39F74019EA9
:102C4B00401F90F40012001EE493FC90064E1200FD
:102C5B001EECF0780A740126F6500418E436F65090
:102C6B00D475F51175D940D2AF22C2AF75D90075A5
:102C7B00F522750A00750900AE09AF0A74FFC39FF0
:102C8B0074019E401F90E60012001EE493FC90001E
:102C9B004E12001EECF0780A740126F6500418E46C
:102CAB0036F650D4750A00750900AE09AF0A74FFE9
:102CBB00C39F74019E401F90E80012001EE493FC1A
:102CCB0090024E12001EECF0780A740126F65004A6
:102CDB0018E436F650D4750A00750900AE09AF0A30
:102CEB0074FFC39F74019E401F90EA0012001EE404
:102CFB0093FC90044E12001EECF0780A740126F639
:102D0B00500418E436F650D4750A00750900AE0964
:102D1B00AF0A74FFC39F74019E401F90EC0012001A
:102D2B001EE493FC90064E12001EECF0780A740120
:102D3B0026F6500418E436F650D475F51175D940C3
:102D4B00D2AF22C2AF75D90075F522750A0075098D
:102D5B0000AE09AF0A74FFC39F74019E401F90DE43
:102D6B000012001EE493FC90004E12001EECF07853
:102D7B000A740126F6500418E436F650D4750A008E
:102D8B00750900AE09AF0A74FFC39F74019E401F03
:102D9B0090E00012001EE493FC90024E12001EEC19
:102DAB00F0780A740126F6500418E436F650D47500
:102DBB000A00750900AE09AF0A74FFC39F74019E28
:102DCB00401F90E20012001EE493FC90044E120090
:102DDB001EECF0780A740126F6500418E436F6500F
:102DEB00D4750A00750900AE09AF0A74FFC39F744E
:102DFB00019E401F90E40012001EE493FC90064ECF
:102E0B0012001EECF0780A740126F6500418E43612
:102E1B00F650D475F51175D940D2AF22C2AF75D922
:102E2B000075F522750A00750900AE09AF0A74FF2B
:102E3B00C39F74019E401F90D60012001EE493FCAA
:102E4B0090004E12001EECF0780A740126F6500426
:102E5B0018E436F650D4750A00750900AE09AF0AAE
:102E6B0074FFC39F74019E401F90D80012001EE494
:102E7B0093FC90024E12001EECF0780A740126F6B9
:102E8B00500418E436F650D4750A00750900AE09E3
:102E9B00AF0A74FFC39F74019E401F90DA001200AB
:102EAB001EE493FC90044E12001EECF0780A7401A1
:102EBB0026F6500418E436F650D4750A007509004E
:102ECB00AE09AF0A74FFC39F74019E401F90DC00D4
:102EDB0012001EE493FC90064E12001EECF0780AD2
:102EEB00740126F6500418E436F650D475F51175B6
:102EFB00D940D2AF22E51464046006E59964FF6003
:102F0B00028031A20E4004D20E8027E514600874B3
:102F1B00E62514900023F0E513600874F025139058
:102F2B000023F0E514B4010280FE75140075130044
:102F3B00C20E8002C20EE514903861F82828737512
:102F4B001400E599B4FF03751301E599B4FE0375FD
:102F5B001302E599B4FD03751303E599B4FC0375EE
:102F6B001304E599B4FA03751305E599B4FB0675DB
:102F7B001401120464E599B4F9067514041204647F
:102F8B00E599D394E54007E599C394F04002801688
:102F9B008599157514027E017F00E515C394E61221
:102FAB003F4D8E0D8F0E900786E4F0A3F0E599D37D
:102FBB0094C44007E599C394E6400280288599158F
:102FCB0075140374E5C39515F50E750D00AE0DAFB5
:102FDB000E9038BE12002EE493F87401939007867E
:102FEB00C8F0A3C8F0D299023475900786E0FEA30F
:102FFB00E0FFEFC39400EE94054009EFD394FFEE8E
:10300B0094064013900786E0FEA3E0FF90004E125B
:10301B00001EE599F0800385996B90078612000ED0
:10302B00900786E0FEA3E0FFEFB40106EEB40702C3
:10303B00800302328290074EE0B43C0280030232DE
:10304B008275FFA0A20AB35005A20BB34003023155
:10305B0075C29C90007AE090078CF0900057E0903E
:10306B00078DF0900062E090078EF0900063E09087
:10307B00078FF0900074E0900790F090007CE09048
:10308B000791F090007DE0900792F0900080E09027
:10309B000793F0900081E0900794F090013AE09054
:1030AB000795F090013BE0900796F090013CE09083
:1030BB000797F0900090E0900798F0900091E090C7
:1030CB000799F0900092E090079AF0900093E090AF
:1030DB00079BF0900094E090079CF0900095E09097
:1030EB00079DF0900096E090079EF0900097E0907F
:1030FB00079FF0900099E09007A0F090009AE09065
:10310B0007A1F090009BE09007A2F090009CE0904C
:10311B0007A3F07400900082F01200AC74AB900720
:0D312B0088F01225F974AA900788F0E55786
:06386100022F4A022FF5C0
:10313800903882F828287380121226A4800D12274E
:0B314800E280081229208003122A5E9A
:0F38820002313F02314102314602314B023150D7
:10315300900788E4F090013AE0700C90013BE07036
:103163000690013CE060028004C20A8002D20A0297
:103173003277C29C900078E0900789F090005EE07F
:1031830090078AF090005FE090078BF090007AE060
:1031930090078CF0900057E090078DF0900062E06C
:1031A30090078EF0900063E090078FF0900074E03A
:1031B300900790F090007CE0900791F090007DE004
:1031C300900792F0900080E0900793F0900081E0E8
:1031D300900794F090013AE0900795F090013BE05E
:1031E300900796F090013CE0900797F0900090E0F4
:1031F300900798F0900091E0900799F0900092E08A
:1032030090079AF0900093E090079BF0900094E071
:1032130090079CF0900095E090079DF0900096E059
:1032230090079EF0900097E090079FF0900099E040
:103233009007A0F090009AE09007A1F090009BE027
:103243009007A2F090009CE09007A3F07400900018
:1032530082F074AB900788F01225F974AA9007885E
:10326300F01226A41227E2122920122A5ED29C759C
:1032730099FB80FED29C7514007513007599FB02AF
:103283003475900786E0FEA3E0FFEF4E7006859944
:1032930010750F00900786E0FEA3E0FF74016F4EE8
:1032A300701BAC0FAD10AA0DAB0EED2BFBEC3AFA75
:1032B3008A068B0790004E12001EE599F090078650
:1032C30012000E900786E0FEA3E0FF74026F4E70BB
:1032D3000C1200AC85159975140075130002347532
:1032E300900786E0FEA3E0FF90004E12001EE599D2
:1032F300F090078612000E900786E0FEA3E0FFAC75
:103303000DAD0E8F028E038C068D079038F61200DA
:103313002EE493F9740193FEEAD39EEB9940098559
:103323001599751400751300023475900786E0FE35
:10333300A3E0FF90004E12001EE599F0900786125D
:10334300000E900786E0FEA3E0FFEFB40006EEB4A4
:103353000102800302347575FFA090001CE0D39432
:10336300C7400B90001CE0C394C8F516801A900068
:103373001CE0D39463400B90001CE0C39464F516E7
:10338300800690001CE0F516E51675F002A4FFAE6A
:10339300F08F6AEF90004E123F65EFFCE0FDEC907A
:1033A3000051123F65EDFCE0FDEC2DB516028003E4
:1033B3000234670FEF90004E123F65E56AFFE0FCB1
:1033C300EF900052123F65ECFFE0FCEFC39CB51693
:1033D300028003023467E56A900050123F65E56A94
:1033E300FFE0FCEF900053123F65ECFFE0FCEF2C95
:1033F300B51671E56A900054123F65E0C3951690C7
:10340300079DF0E56A900055123F65E0C39516905D
:10341300079EF0E56A900058123F65E0C395169049
:10342300079FF0E56A900059123F65E0C395169037
:1034330007A0F0E56A90005A123F65E0C395169025
:1034430007A1F0E56A90005B123F65E0C395169013
:1034530007A2F012256F7599F97518647517001294
:10346300252B80FE7599FF75186475170012252B9F
:0234730080FED9
:093867000232850232E302332E25
:1034750022E513903870F82828730235B690078630
:10348500E0FEA3E0FF90001212001EE0F599900700
:103495008612000E900786E0FEA3E0FF74116F4EC2
:1034A50070037513000235B68561990235B690072C
:1034B50086E0FEA3E0FF90004E12001EE0F599EFB6
:1034C500B40107EEB4070375130090078612000ECA
:0734D5000235B6900787E005
:0F38700002347F0234820234AD0234B30234D802
:1034DC00903891F82828738523990235AB85299962
:1034EC000235AB8543990235AB8546990235AB85E0
:1034FC0050990235AB855F990235AB8555990235EC
:10350C00AB8557990235AB756D00900069E070067C
:10351C00900068E060028016A2A44006E56D4404A9
:10352C00F56DA2A54006E56D4402F56D801A90007C
:10353C004AE0B40106E56D4410F56D900049E0B425
:10354C000106E56D4420F56DA207B34006E56D4418
:10355C0001F56DA209B34006E56D4408F56D856D66
:10356C0099803CA20FB340077599FAC20F8017A23D
:10357C000CB3400575990F800B900023E0F59990E2
:10358C000023E4F0C20C80178541998012854A997A
:0F359C00800D85459980087599FC800375130093
:103891000234E30234E90234EF0234F50234FB026C
:1038A100350102350702350D02351302356F023538
:0D38B1009402359902359E0235A30235A818
:0B35AB0090078612000E8003120048FB
:03387F000235B35C
:1035B6002290006BE0B4010385231190006BE0B408
:1035C600020385291190006BE0B403038543119033
:1035D600006BE0B4040385461190006BE0B405036C
:1035E60085501190006BE0B4060385551190006B71
:1035F600E0B4070385571190006CE0FE90006DE083
:10360600C39E500302368D90006BE0D39404402C89
:1036160090006CE0D39511500990006DE0C39511B0
:1036260050028002D20090006CE0D39511500990B0
:10363600006DE0C395115002C200804990006BE016
:10364600B4041890006DE0C395115002D2009000AA
:103656006CE0D395114002C200802A90006CE0C352
:103666009511500990006DE0D3951150028002D259
:103676000090006CE0D39511500990006DE0C39561
:10368600115002C200807E90006BE0D39404402C5F
:1036960090006CE0C39511400990006DE0D3951140
:1036A60040028002C20090006CE0C3951140099070
:1036B600006DE0D395114002D200804990006BE086
:1036C600B4041890006CE0C395115002C20090003B
:1036D6006DE0D395114002D200802A90006CE0C3C1
:1036E6009511400990006DE0D395114002D20090EB
:1036F600006CE0D39511400990006DE0C395114030
:10370600028002C2002290006EE0B40103852311FC
:1037160090006EE0B4020385291190006EE0B403B8
:103726000385431190006EE0B404038546119000B2
:103736006EE0B4050385501190006EE0B406038573
:10374600551190006EE0B4070385571190006FE0A5
:10375600FE900070E0C39E50030237E290006EE0D8
:10376600D39404402C90006FE0D39511500990003B
:1037760070E0C3951150028002D20290006FE0D330
:1037860095115009900070E0C395115002C2028055
:103796004990006EE0B40418900070E0C395115093
:1037A60002D20290006FE0D395114002C202802A35
:1037B60090006FE0C395115009900070E0D3951109
:1037C60050028002D20290006FE0D395115009900A
:1037D6000070E0C395115002C202807E90006EE038
:1037E600D39404402C90006FE0C3951140099000DB
:1037F60070E0D3951140028002C20290006FE0C3D0
:1038060095114009900070E0D395114002D20280D4
:103816004990006EE0B4041890006FE0C395115013
:1038260002C202900070E0D395114002D202802AB3
:1038360090006FE0C395114009900070E0D3951198
:103846004002D20290006FE0D395114009900070BB
:0B385600E0C3951140028002C2022274
:093F65002582F582500205832239
:10002E00EF2F500205832582F582E5833E2EF58360
:01003E00229F
:08000300C3EF9DFFEE9CFE22FD
:08003F000806B60002180622B3
:0D000E00A3E004F07006123F5BE004F02256
:083F77000816B6FF021816221D
:0E3F3F00048007C3CE13CECF13CFD5E0F622F9
:103DED00BC000FBE0008ED8FF084FFADF022E4FEA5
:103DFD00FF22BE000DEF60FE54F0606F20E703025E
:103E0D003EA3EAC0E0EBC0E078017A0075F001EE68
:103E1D0020E710EF25E0FFEE33FE0AC5F023C5F0D5
:103E2D0030E7F0EA5407F9096A7A007B006001086F
:103E3D00C3EC9E40167004ED9F4010ED9FFDEC9E6F
:103E4D00FCE5F0CA4ACA03F5F08005E5F003F5F08C
:103E5D00C3EE13FEEF13FFD9D77908CACBCAD8D05A
:103E6D00EAFEEBFFD0E0FBD0E0FA22EC8FF084FC11
:103E7D00ED54F045F0C48FF084FEEDC454F045F0E0
:103E8D00C48FF084FDEEC4FE54F02DFFEE540F3CB4
:103E9D00FEADF07C0022790078008FF0EC7E0820DA
:103EAD00E70DC3CD33CD33C933C9C833C8DEF08474
:103EBD0049F9E5F08FF0BE00E6FD7C00E9FFE8FE74
:013ECD0022D2
:0E3F4D00F88FF0A4FFE5F0CE88F0A42EFE223F
:103F1F00600D782B023F29007830D8FED5E0F822CB
:103F2F00EEC0E07E00123DEDEFFDEEFCD0E0FE2294
:03000B00023ECEE4
:03001B00023EE9B9
:03002B00023F048D
:03000000023F6E4E
:093F6E0075817175D0000206FF97
:0B001E00E5822FF582E5833EF583228A
:0A3F5B000582D5820215831582222B
:103ECE00C0E0C0F0C083C082C0D075D0001206F42E
:103EDE00D0D0D082D083D0F0D0E032C0E0C0F0C0DD
:103EEE0083C082C0D075D0001206F7D0D0D082D059
:103EFE0083D0F0D0E032C0E0C0F0C083C082C0D02A
:103F0E0075D0001206FAD0D0D082D083D0F0D0E097
:013F1E003270
:00000001FF
